:0200000480007A
:100000006F000005732F2034930F80006308FF03F7
:10001000930F90006304FF03930FB0006300FF038E
:10002000130F000063040F0067000F00732F2034CC
:1000300063540F006F00400093E19153171F0000BD
:1000400023223FFC171F000023200FFC6FF01FFF2F
:100050009300000013010000930100001302000050
:100060009302000013030000930300001304000038
:100070009304000013050000930500001306000020
:100080009306000013070000930700001308000008
:10009000930800001309000093090000130A0000F0
:1000A000930A0000130B0000930B0000130C0000D8
:1000B000930C0000130D0000930D0000130E0000C0
:1000C000930E0000130F0000930F0000732540F102
:1000D0006310050097020000938202017390523072
:1000E000735044749702000093820201739052305F
:1000F00073500018970200009382020273905230EE
:10010000B70200809382F2FF7390023B9302F001EA
:100110007390023A7350403097020000938242017C
:100120007390523073502030735030309301000080
:1001300097020000938242ED739052301305100035
:100140001315F501634C05000F00F00F930110002B
:100150009308D0051305000073000000930200000F
:10016000638A020073905210B7B20000938292101B
:100170007390223073500030970200009382420146
:1001800073901234732540F173002030172400005F
:10019000130444E793011000130310208313140089
:1001A000631C735293012000130310208353140027
:1001B00063147352930130003703030413031320B5
:1001C00083231400631A735093014000370304051E
:1001D00013032330832324006310735093015000D2
:1001E0003703050613033340832334006316734E2D
:1001F00093010001372300001303F3018313F4017B
:10020000631C734C93011001372300001303F301A7
:100210008353F4016312734C9301200137231F2091
:100220001303D3E18323D4016318734A930130018C
:10023000372320211303E3F18323E401631E734872
:1002400093014001372321221303F3018323F40197
:10025000631473489301F001374300001303F30361
:100260008313F403631A73469301000237430000BB
:100270001303F3038353F4036310734693011002D3
:1002800037433F401303D3E38323D40363167344FC
:1002900093012002374340411303E3F38323E40334
:1002A000631C734293013002374341421303F3034B
:1002B0008323F403631273429301E0023783FFFF49
:1002C00013030318A3106400831314006316734010
:1002D0009301F0023783000013032338A310640056
:1002E00083531400631A733E930100033783868798
:1002F00013034358A320640083231400631E733C3C
:100300009301100337938A8B13038398232164008E
:10031000832324006312733C9301200337938E8F51
:100320001303C3D8A3216400832334006316733AF4
:100330009301D00337D3FFFF1303435DA31F640072
:100340008313F401631A73389301E00337D3000079
:100350001303637DA31F64008353F401631E73368C
:100360009301F00337E3DADB1303839DA32E6400CC
:100370008323D401631273369301000437E3DEDF75
:100380001303C3DD232F64008323E4016316733456
:100390009301100437E3E2E31303031EA32F640069
:1003A0008323F401631A73329301C00437330000CE
:1003B00013034353A31F64028313F403631E7330B8
:1003C0009301D0043733000013036373A31F640247
:1003D0008353F403631273309301E00437433A3BD1
:1003E00013038393A32E64028323D4036316732E13
:1003F0009301F00437433E3F1303C3D3232F64021A
:100400008323E403631A732C9301000537434243AB
:1004100013030314A32F64028323F403631E732ABC
:100420009301B00537A3000013038399930380F968
:10043000A3106400030E14006390C32B9301C00546
:1004400037A300001303A3B99303B0F9A31064000A
:10045000030E24006392C3299301D00537A3000043
:100460001303C3D99303C009A3106400034E1400FF
:100470006394C3279301E00537A300001303E3F956
:100480009303F009A3106400034E24006396C32570
:100490009301F00537A3A2A31303031A930300FAF1
:1004A000A3206400030E14006398C3239301000685
:1004B00037A3A6A71303435A9303500A23216400CA
:1004C000034E3400639AC3219301100637B3AAABDD
:1004D0001303839AB7B3FFFF938393AAA321640006
:1004E000031E4400639AC31F9301200637B3AEAFC7
:1004F0001303C3DAB7B300009383E3FAA3216400C4
:10050000035E5400639AC31D9301A00637F30000F5
:100510001303839E930380FEA31F6400030EF40164
:10052000639CC31B9301B00637F300001303A3BE03
:100530009303B0FEA31F6400030E0402639EC3195D
:100540009301C00637F300001303C3DE9303C00E0C
:10055000A31F6400034EF4016390C3199301D006F6
:1005600037F300001303E3FE9303F00EA31F6400B0
:10057000034E04026392C3179301E00637F3F2F3CC
:100580001303031F930300FFA32E6400030ED40183
:100590006394C3159301F00637F3F6F71303435F33
:1005A0009303600F232F6400034E04026396C3136A
:1005B000930100073703FBFB1303839F9303A0BF43
:1005C000A32E6400031EF4016398C3119301100766
:1005D0003703FFFF1303C3DFB70301009383C3DFB8
:1005E000A32F6400035EF4016398C30F9301900787
:1005F000375300001303839493038004A31F640202
:10060000030EF403639AC30D9301A0073753000050
:100610001303A3B49303B004A31F6402030E0404E2
:10062000639CC30B9301B007375300001303C3D47B
:100630009303C004A31F6402034EF403639EC30923
:100640009301C007375300001303E3F49303F0044E
:10065000A31F6402034E04046390C3099301D007EF
:10066000375352531303031593030005A32E64025B
:10067000030ED4036392C3079301E0073753565721
:100680001303435593036005232F6402034E0404B0
:100690006394C3059301F00737635A5B1303839593
:1006A000B76300009383A3B5A32E6402031EF40373
:1006B0006394C3039301000837635E5F1303C3D5DC
:1006C000B76300009383C3D5A32F6402035EF403D2
:1006D0006394C301631030020F00F00F63800100C8
:1006E0009391110093E111009308D0051385010047
:1006F000730000000F00F00F930110009308D00565
:100700001305000073000000731000C0000000001B
:1007100000000000000000000000000000000000D9
:1007200000000000000000000000000000000000C9
:0C073000000000000000000000000000BD
:1010000000000000000000000000000000000000E0
:1010100000000000000000000000000000000000D0
:1010200000000000000000000000000000000000C0
:1010300000000000000000000000000000000000B0
:081040000000000000000000A8
:10200000000102030405060708090A0B0C0D0E0F58
:10201000101112131415161718191A1B1C1D1E1F48
:10202000202122232425262728292A2B2C2D2E2F38
:10203000303132333435363738393A3B3C3D3E3F28
:10204000404142434445464748494A4B4C4D4E4F18
:10205000505152535455565758595A5B5C5D5E5F08
:10206000606162636465666768696A6B6C6D6E6FF8
:10207000707172737475767778797A7B7C7D7E7FE8
:102080005050505050505050505050505050505050
:102090005050505050505050505050505050505040
:1020A0005050505050505050505050505050505030
:1020B0005050505050505050505050505050505020
:1020C0005050505050505050505050505050505010
:1020D0005050505050505050505050505050505000
:1020E00050505050505050505050505050505050F0
:1020F00050505050505050505050505050505050E0
:1021000050505050505050505050505050505050CF
:1021100050505050505050505050505050505050BF
:1021200050505050505050505050505050505050AF
:10213000505050505050505050505050505050509F
:10214000505050505050505050505050505050508F
:10215000505050505050505050505050505050507F
:10216000505050505050505050505050505050506F
:1021700050505050505050505050505050505000AF
:040000058000000077
:00000001FF
